:100000000C942A001895000018950000189500001F
:10001000189500001895000018950000189500002C
:10002000189500001895000018950000189500001C
:10003000189500001895000018950000189500000C
:1000400018950000189500001895000018950000FC
:10005000189500008FE58DBFC8E3E0E24E2E84E0E6
:100060008EBFD4E0F4E05F2EA89584B7082E877F7A
:1000700084BF88E1992781BD91BDEEEFF3E0A0E652
:10008000B0E088278D933197E9F766248FEF81BB25
:100090008FE38093600086E0809361008BE580931E
:1000A00062008FE48093630086E6809364008DE6AF
:1000B000809365008DEF8093660087E080936700F2
:1000C0008FE7809368008FE68093690080E090E07E
:1000D000AAE6B0E08D939C93AAE6B0E00D911C9146
:1000E000093050E015071CF011F00C948E00AAE6C0
:1000F000B0E0AD90BD90A0E6B0E0AA0DBB1DE2E37C
:10010000F0E08C918095808384EF91E00E94A200C2
:10011000AAE6B0E00E9492000C946C000C94660079
:10012000F894FFCFED91FC91EF5FFF4FFC93EE93BE
:1001300008953197F1F70895689462F80895E89466
:1001400062F80895EF93FF93EE27E82BE92B31F047
:10015000E0EAFFE03197F1F70197D1F7FF91EF91D6
:02016000089500
:00000001FF
